:1008000050EF04F0FF00FF00D9CF6EF0DACF6FF0A9
:10081000F3CF70F08BEF23F0D8CF4EF0E8CF4FF04E
:10082000E0CF50F0E1CF51F0E2CF52F0D9CF53F00A
:10083000DACF54F0F3CF55F0F4CF56F0F6CF57F0AF
:10084000F7CF58F0F8CF59F0F5CF5AF0010EF2A4D7
:10085000000EF2AA000EE8A003D04D6A4D2A01D086
:100860004D6A4D50D8A416EC11F05AC0F5FF59C08E
:10087000F8FF58C0F7FF57C0F6FF56C0F4FF55C049
:10088000F3FF54C0DAFF53C0D9FF52C0E2FF51C09A
:10089000E1FF50C0E0FF4FC0E8FF4EC0D8FF10009E
:1008A000F5EF22F04C6EEF0E176EFF0E186E4C50E7
:1008B000D96EDA6ADECF19F0DECF1AF0DECF1BF088
:1008C000DECF1CF03CEC09F045D14C5024EF0EF08B
:1008D000D1D909E15151491806E152514A1803E1B1
:1008E00053514B18D8A41200D8EF21F0C3D909E115
:1008F0005151491806E152514A1803E153514B181E
:10090000D8A412004C50D96EFEEC0CF002E19CEF22
:100910001EF04C50ADEF21F0ADD90BE1515149180B
:1009200008E152514A1805E153514B1802E1E2EF38
:100930001EF04C50D96EDA6ADF50446E3F0E4416FA
:10094000D8A43F0C5CC001F05DC002F039EC24F08B
:1009500001EC22F00D5062EC24F0E2EF1EF08AD997
:1009600009E15151491806E152514A1803E1535126
:100970004B18D8A412004C50B9EF16F07BD909E1FE
:100980005151491806E152514A1803E153514B188D
:10099000D8A41200086AC80E076E010E096E0B6A11
:1009A000C80E0A6E7BD9016E026A030E046EE80E51
:1009B000036E78EC23F001C00CF002C00DF0020EC3
:1009C000E1EC1CF04C5055EF1EF054D909E15151A7
:1009D000491806E152514A1803E153514B18D8A463
:1009E00012004C5041EF10F045D909E1515149181E
:1009F00006E152514A1803E153514B18D8A4120092
:100A00004C50E8EF11F036D909E15151491806E18F
:100A100052514A1803E153514B18D8A412004C50BC
:100A200016EF16F027D909E15151491806E1525144
:100A30004A1803E153514B18D8A412004C5073EFDD
:100A400015F018D909E15151491806E152514A18D7
:100A500003E153514B18D8A412004C50B3EF12F0DD
:100A600009D909E15151491806E152514A1803E1E7
:100A700053514B18D8A412004C50EBEF0BF0FAD89E
:100A800009E15151491806E152514A1803E1535105
:100A90004B18D8A412004C5057EF20F04C50D96E90
:100AA000DA6A0C0ED926DF50446E4C50D96EDA6AE1
:100AB0000B0ED926DF50456E4C50D96EDA6A0A0EFD
:100AC000D926DF50466E4C50D96EDA6A090ED92607
:100AD000DF50476E4C50D96EDA6A080ED926DF50C7
:100AE000486E4C50D96EDA6A070ED926DF50496E2F
:100AF0004C50D96EDA6A060ED926DF504A6ECED82F
:100B00004A244924482447244624452444240001F7
:100B1000B26F460EB219D8A41200ACD809E15151F7
:100B2000491806E152514A1803E153514B18D8A411
:100B30001200F29EC4EF1DF001014C5107E1E5ECFB
:100B40001BF0000E0D6A0C6AE1EC1CF0500E010166
:100B50004C6F500C4C50D96EDA6A000EDE14446EA5
:100B6000FC0EDE14456EFF0EDE14466E1F0EDE1404
:100B7000476E47506CE0020A6EE00A0A71E0120A02
:100B8000D8A4120072D04550D8A412004450D8A462
:100B900012009BD645501AE0040A1CE00C0A1EE025
:100BA000040A20E01C0A22E0040A24E00C0A26E0E1
:100BB000040A26E02C0A28E0040A2AE00C0A2CE0A9
:100BC000780A2EE0040AD8A412002ED04450D8A4EB
:100BD0001200FBD64450D8A4120024D74450D8A405
:100BE000120002D74450D8A412002BD74450D8A4E6
:100BF000120009D74450D8A4120041D74450120023
:100C00004450D8A412002CD74450D8A4120060D667
:100C10004450D8A41200A3D64450D8A4120066D6DB
:100C20004450D8A41200AAD64450D8A4120074D6B6
:100C300045501C0AD8A412004450D8A412007CD7F6
:100C40004550D8A412004450D8A4120027D74650CB
:100C5000D8A4120098D74650070AD8A412009AD7F1
:100C60004650040AD8A41200E3D74650070AD8A475
:100C70001200E6D74C50D96EDA6ADECF44F0DECFF0
:100C800045F0DECF46F0DECF47F03F0E4414486E0D
:100C9000496A4A6A4B6A0101501912004C50D96ED8
:100CA000DA6A050ED926DF5012008A0E9F6F20D116
:100CB000250EA51904E0A55141EC24F019D1A46B2F
:100CC00037D0A48935D0A48F47D09F51D96EDA6A26
:100CD000DECF9DF0DDCF9EF0020E9F279D519E112D
:100CE00015E1E80E9D6FFF0E9E6F10D052D9F7648C
:100CF00003D00800F55005D0F6CFE1FFF7CFE2FFB3
:100D0000E75041EC24F000019D4B9E2B42D9F76443
:100D100003D00800F55005D0F6CFE1FFF7CFE2FF92
:100D2000E750000901E1E4D0E1D7C00EA41314D0CC
:100D300088C0F6FF89C0F7FF24D9D8B41200640A2E
:100D40000BE00D0A09E0050ABCE01F0ABEE0060A36
:100D5000ECE00D0AB8E0CCD0A4C098F0C00E981713
:100D60001FE1A4A902D0E1D80DD09F51D96EDA6A53
:100D7000DECFA0F0DDCFA1F0000EA1BFFF0EA26F6D
:100D8000A36F020E9F27A3AF4BD0030EA413A31F84
:100D9000A21FA11FA06D000EA123A223A32340D058
:100DA000A4A902D0C2D80ED09F51D96EDA6ADECF84
:100DB00098F0DDCF99F098C0A0F099C0A1F0A26B97
:100DC000A36B020E9F272CD0010EA56FA5519FD8B3
:100DD00098D8F550A05D0900F550A1590900F550CB
:100DE000A2590900F550A35922E3A52B0A0EA51913
:100DF0001EE0ECD7010EA56FA55190D882D8F55012
:100E0000A05D0900F550A1590900F550A25909004B
:100E1000F550A3590CE3A52B080EA51908E0ECD753
:100E2000A451C00BD1E0800AE5E0400ACDE0A4C0A7
:100E300098F0030E981703E02D0E41EC24F000010A
:100E4000A5519B6F9C6B9BBF9C074AD086D8A50E73
:100E50009825F66EFE0E992154D873D8A0C072F072
:100E6000A1C073F0A2C074F0A3C075F0E1EC1FF054
:100E700072C07FF073C080F074C081F075C082F0E2
:100E80000A0E836F846B856B866BC1EC20F07F51FB
:100E9000300FA56F22D0A0C072F0A1C073F0A2C025
:100EA00074F0A3C075F059D8CD0E9825F66EFE0EDD
:100EB000992127D846D8E1EC1FF072510F0B9A6F99
:100EC0005E0E9A2555D8F5CFA5F007D0A451C00BDA
:100ED000BDE0800AE0E0400AB9E0A55141EC24F011
:100EE00000019B07D8A09C079B29F0E19C29EEE11B
:100EF00088C0F6FF89C0F7FF000143D8D8B41200BC
:100F0000D7D6F76EF86A000EF82209001200040D19
:100F1000A50EF324F66EFE0EF4201200040DCD0E85
:100F2000F324F66EFE0EF42012009F51D96EDA6A99
:100F3000DECFA0F0DECFA1F0DECFA2F0DECFA3F0B7
:100F4000040CF5CF76F00900F5CF77F00900F5CF66
:100F500078F00A00F5CF79F012009BC098F09CC0A1
:100F600099F0D89098379937D890983799371200D8
:100F7000F66EF76AFF0EF722F86A000EF8220800F4
:100F80001200884B892BF86A0800F5CFA5F0A5510F
:100F900012009DC0F6FF9EC0F7FF000EF86E0E0E09
:100FA00012007F6F0F0120B72ED0210E0001726F4B
:100FB0000F0E1AD96DEC1AF07F51D96EFEEC0CF0C1
:100FC0000F01256F20D90F01266F000132D90F01C3
:100FD000276F000135D90F01286F000146D90F0195
:100FE000296F00013BD90F012A6F00011BD90F01A6
:100FF0002B6F00012CD90F012C6F00010CD90F01B0
:101000002D6F2087120010B72ED0110E0001726FC5
:101010000F0EEAD86DEC1AF07F51D96EFEEC0CF091
:101020000F01156FF0D80F01166F000102D90F01E3
:10103000176F000105D90F01186F000116D90F01B4
:10104000196F00010BD90F011A6F0001EBD80F01C6
:101050001B6F0001FCD80F011C6F0001DCD80F01D1
:101060001D6F1087120000B72ED0010E0001726FA5
:101070000F0EBAD86DEC1AF07F51D96EFEEC0CF061
:101080000F01056FC0D80F01066F0001D2D80F0104
:10109000076F0001D5D80F01086F0001E6D80F01D6
:1010A000096F0001DBD80F010A6F0001BBD80F01E7
:1010B0000B6F0001CCD80F010C6F0001ACD80F01F1
:1010C0000D6F008712000E01B0B72ED0B10E0001D7
:1010D000726F0E0E89D86DEC1AF07F51D96EFEEC4E
:1010E0000CF00E01B56F8FD80E01B66F0001A1D8BC
:1010F0000E01B76F0001A4D80E01B86F0001B5D87A
:101100000E01B96F0001AAD80E01BA6F00018AD88A
:101110000E01BB6F00019BD80E01BC6F00017BD894
:101120000E01BD6FB0871200C0B72ED0C10E0001F6
:10113000726F0E0E59D86DEC1AF07F51D96EFEEC1D
:101140000CF00E01C56F5FD80E01C66F000171D89B
:101150000E01C76F000174D80E01C86F000185D859
:101160000E01C96F00017AD80E01CA6F00015AD86A
:101170000E01CB6F00016BD80E01CC6F00014BD874
:101180000E01CD6FC0871200D0B71200D10E000142
:10119000726F0E0E29D86DEC1AF07F51D96EFEECED
:1011A0000CF00E01D56F2FD80E01D66F000141D87B
:1011B0000E01D76F000144D80E01D86F000155D839
:1011C0000E01D96F00014AD80E01DA6F00012AD84A
:1011D0000E01DB6F00013BD80E01DC6F00011BD854
:1011E0000E01DD6FD0871200736F7F51D96EDA6AFE
:1011F000DECF74F0DECF75F0DECF76F0DECF77F0A5
:101200007EC078F0120000017F51D96EDA6A050EB7
:10121000D926DF5012007F51D96EDA6A0C0ED9261A
:10122000DF5012007F51D96EDA6A0A0ED926DF50DC
:1012300012007F51D96EDA6A060ED926DF501200ED
:101240007F51D96EDA6A070ED926DF5012007F511E
:10125000D96EDA6A0B0ED926DF5012007F51D96E93
:10126000DA6A090ED926DF5012007F51D96EDA6A88
:10127000080ED926DF501200190E2E6E20D1250E31
:10128000341804E0345068EC24F019D1336A36D0B5
:10129000338834D0338E42D02E50D96EDA6ADECF06
:1012A0002CF0DDCF2DF0020E2E262C502D1014E147
:1012B000E80E2C6EFF0E2D6E0FD034D9F76403D0DC
:1012C0000800F55005D0F6CFE1FFF7CFE2FFE75079
:1012D00068EC24F02C4A2D2A25D9F76403D00800A5
:1012E000F55005D0F6CFE1FFF7CFE2FFE750000958
:1012F00001E1E5D0E2D7C00E331210D0FCD8D8B44B
:101300001200640A0BE00D0A09E0050AC1E01F0A99
:10131000C3E0060AF0E00D0ABDE0D1D033C027F0EB
:10132000C00E27161FE133A802D0CDD80DD02E5005
:10133000D96EDA6ADECF2FF0DDCF30F0000E30BE8E
:10134000FF0E316E326E020E2E2632AE4FD0030EDD
:101350003312321E311E301E2F6C000E302231220D
:10136000322244D033A802D0AED80ED02E50D96E3F
:10137000DA6ADECF27F0DDCF28F027C02FF028C0B3
:1013800030F0316A326A020E2E2630D0010E346EF1
:10139000345087EC07F081EC07F0F5502F5C090022
:1013A000F55030580900F55031580900F5503258C1
:1013B00024E3342A0A0E341820E0EAD7010E346EF2
:1013C00034508EEC07F081EC07F0F5502F5C0900EB
:1013D000F55030580900F55031580900F550325891
:1013E0000CE3342A080E341808E0EAD73350C00B57
:1013F000CDE0800AE3E0400AC9E033C027F0030EE5
:10140000271603E02D0E68EC24F034502A6E2B6A68
:101410002ABE2B064DD07BD8A50E2724F66EFE0ED5
:10142000282081EC07F05BD82FC001F030C002F01B
:1014300031C003F032C004F01CEC20F001C00EF00B
:1014400002C00FF003C010F004C011F00A0E126EBB
:10145000136A146A156AF2EC20F00E50300F346EE5
:1014600024D02FC001F030C002F031C003F032C0F0
:1014700004F04DD8CD0E2724F66EFE0E282081EC08
:1014800007F02DD81CEC20F001500F0B296E5E0EDA
:101490002924B8EC07F0F5CF34F007D03350C00B57
:1014A000BAE0800ADEE0400AB6E0345068EC24F08E
:1014B0002A06D8A02B062A28F1E12B28EFE11BD819
:1014C000D8B41200DCD62E50D96EDA6ADECF2FF0F7
:1014D000DECF30F0DECF31F0DECF32F0040CF5CFCE
:1014E00005F00900F5CF06F00900F5CF07F00A0076
:1014F000F5CF08F0120017C0F6FF18C0F7FF174A23
:10150000182AF86A0800F5CF34F0345012002AC0C7
:1015100027F02BC028F0D89027362836D8902736C9
:10152000283612002CC0F6FF2DC0F7FF000EF86E13
:101530000E0E1200E0D0610E606F0F0EF8D856EC60
:1015400018F0B15110D965CFDFFFB15114D966CF72
:10155000DFFFB15100D967CFDFFFB151F4D868CFB9
:10156000DFFFB15118D969CFDFFFB1510CD96ACF74
:10157000DFFFB15120D96BCFDFFFB15114D96CCF50
:10158000DFFFB15120D96DCFDFFF609EC8D0310E93
:10159000606F0F0ECCD856EC18F0B151E4D835CFAF
:1015A000DFFFB151E8D836CFDFFFB151D4D837CF04
:1015B000DFFFB151C8D838CFDFFFB151ECD839CFF8
:1015C000DFFFB151E0D83ACFDFFFB151F4D83BCFC4
:1015D000DFFFB151E8D83CCFDFFFB151F4D83DCFA8
:1015E000DFFF0F01309F9BD0810E606F0E0E9FD8E2
:1015F00056EC18F0B151B7D885CEDFFFB151BBD84A
:1016000086CEDFFFB151A7D887CEDFFFB1519BD87F
:1016100088CEDFFFB151BFD889CEDFFFB151B3D83B
:101620008ACEDFFFB151C7D88BCEDFFFB151BBD817
:101630008CCEDFFFB151C7D88DCEDFFF0E01809F6A
:101640006ED0910E606F0E0E72D856EC18F0B1513C
:101650008AD895CEDFFFB1518ED896CEDFFFB1513B
:101660007AD897CEDFFFB1516ED898CEDFFFB15157
:1016700092D899CEDFFFB15186D89ACEDFFFB15113
:101680009AD89BCEDFFFB1518ED89CCEDFFFB151EF
:101690009AD89DCEDFFF0E01909F41D0A10E606FC2
:1016A0000E0E45D856EC18F0B1515DD8A5CEDFFF2F
:1016B000B15161D8A6CEDFFFB1514DD8A7CEDFFF23
:1016C000B15141D8A8CEDFFFB15165D8A9CEDFFF17
:1016D000B15159D8AACEDFFFB1516DD8ABCEDFFFE3
:1016E000B15161D8ACCEDFFFB1516DD8ADCEDFFFC7
:1016F0000E01A09F14D06F500F0B00016C6F6D6B2B
:101700006D510DE16C5101E116D7010A01E13FD79E
:10171000030A01E169D7010A94E0070ABFE000016A
:10172000B12B0F0EB117B02BB01777920F0C616F62
:10173000B1510D0D000EF324626F020EF420636FA1
:10174000010E646F010C0D0D070EF324D96E020E0D
:10175000F420DA6E12000D0D060EF324D96E020E7F
:10176000F420DA6E12000D0D040EF324D96E020E71
:10177000F420DA6E12000D0D050EF324D96E020E60
:10178000F420DA6E12000D0D090EF324D96E020E4C
:10179000F420DA6E12000D0D080EF324D96E020E3D
:1017A000F420DA6E12000D0D0B0EF324D96E020E2A
:1017B000F420DA6E12000D0D0A0EF324D96E020E1B
:1017C000F420DA6E12000D0D0C0EF324D96E020E09
:1017D000F420DA6E12001A6E1A50D96EDA6AC00E50
:1017E000DE14146EFF0EDE14156EFF0EDE14166E80
:1017F000FF0EDE14176EC8D01A50D96EFFD80CE059
:1018000002D9036F026A060E016E03C103F0D8EC21
:1018100022F084EC24F0A8D01A50E5D8010E000183
:10182000BA6F03C1BBF019D01A50D96EE7D80BE0DC
:10183000EAD802E0028B01D0029BECD8D8EC22F06F
:1018400084EC24F091D01A50CED8010E0001BA6F6A
:1018500001010239E842070B93D0010E0D6EB60E5E
:1018600037EF0FF01A50D96EC9D80BE0CCD802E090
:10187000028501D00295CED8D8EC22F084EC24F079
:1018800073D01A50B0D8010E0001BA6F01010241A5
:10189000E8423F0B75D01A50D96EB0D80BE0B3D8E0
:1018A00002E0028701D00297B5D8D8EC22F084EC90
:1018B00024F05AD01A5097D8010E0001BA6F0101D6
:1018C0000239E8461F0B5CD01A50D96E97D80BE04E
:1018D0009AD802E0028901D002999CD8D8EC22F073
:1018E00084EC24F041D01A507ED8010E0001BA6F6A
:1018F000010102390F0B44D01A5063EC13F0DF647E
:1019000019D01A50D96EDA6A060ED926DF50116E38
:10191000106A79D81024186E000E1120196E19BEA5
:1019200023D0195002E118041FE318C007F119C0B1
:1019300008F11AD01A5057D8020E0001BA6F07C129
:10194000BBF0010108510001BC6F87D71A50D96E56
:1019500055D80DE058D802E0028D01D0029D5AD82A
:10196000D8EC22F084EC24F01A5055EF1EF01A50F7
:101970003AD8010E0001BA6F01010245E846030B97
:10198000010B0001BB6F69D714C010F015C011F036
:1019900016C012F017C013F01350020AD8A4120098
:1019A0001DD011501C0A04E0010AD8A4120009D06D
:1019B0001050CCE0800A01E11FD7400AD8A41200E1
:1019C00033D7105001E14ED7400A01E164D7C00A75
:1019D00001E17AD7400AD8A412008ED71250070A24
:1019E000D8A41200DED7D96EDA6ADECFB6F0DECF29
:1019F000B7F0DECFB8F0DECFB9F01200DA6A040E2D
:101A0000D926DF5012001A50D96EDA6A050ED9268F
:101A1000DF501200026A040E016E0251FC0B036ECD
:101A200012000101000501E0F5D028EC1FF021EEC5
:101A300017F0DECF31F0DDCF32F02950315E2A5081
:101A4000325A31C027F132C028F10101000E28BFFF
:101A5000FF0E296F2A6F21EE3BF0E4D84FEC22F005
:101A600001C02FF102C030F103C031F104C032F1E6
:101A700021EE3DF0D7D84FEC22F001013351012483
:101A8000336F34510220346F35510320356F365196
:101A90000420366F36BF0ED03651351105E1310EB8
:101AA000335D750E345906E3300E336F750E346FA7
:101AB000356B366B36AF0FD0D00E335D8A0E34598E
:101AC000FF0E3559FF0E365906E2D00E336F8A0EDF
:101AD000346F3569366927512B5D016E28512C59B9
:101AE000026E29512D59036E2A512E59046E21EE92
:101AF0003FF0DECF05F0DDCF06F0000E06BEFF0E94
:101B0000076E086E4FEC22F001C037F102C038F1C9
:101B100003C039F104C03AF127C12BF128C12CF1DF
:101B200029C12DF12AC12EF1010133512F25316E2A
:101B300034513021326E35513121336E36513221DC
:101B4000346E375131240B6E385132200C6E3951BE
:101B500033200D6E3A5134200E6E75EC22F00BC01E
:101B600041F10CC042F10DC043F10EC044F1016AD5
:101B7000C00E026E7F0E036E440E046E41C105F06E
:101B800042C106F043C107F044C108F029EC22F03D
:101B900008E20101416BC00E426F7F0E436F440E9D
:101BA000446F41C101F042C102F043C103F044C19E
:101BB00004F0056AC00E066E7F0E076EC40E086E36
:101BC00029EC22F009E2000E0101416FC00E426FC4
:101BD0007F0E436FC40E446F41C11FF042C120F01D
:101BE00043C121F044C122F093EC1CF01FC00DF161
:101BF00020C00EF10DEC1EF001C007F002C008F08D
:101C0000CCEC14F00DEC1EF001C00FF002C010F08F
:101C100090EF1BF0086A076ACCEC14F0106A0F6AA8
:101C200090EF1BF0DECF01F0DDCF02F0000E02BE20
:101C3000FF0E036E046E27C105F028C106F029C10E
:101C400007F02AC108F01200436EBBD0D70E176E02
:101C5000FF0E186E3CEC09F04350ECEC1BF0040E48
:101C60000101006FFDD8CCEC14F081EF24F0B90E27
:101C7000176EFF0E186E3CEC09F04350ECEC1BF0B5
:101C80000101096B0A6B010E006F6EEF24F0E00E8C
:101C9000176EFF0E186E3CEC09F04350ECEC1BF095
:101CA0000101006BDDD8CCEF14F0230E01014D6F64
:101CB000230CC40E176EFF0E186E3CEC09F07ED09C
:101CC0004350D96EDA6A0C0ED926DF503B6E435072
:101CD000D96EDA6A0B0ED926DF503C6E4350D96EAE
:101CE000DA6A0A0ED926DF503D6E4350D96EDA6AA1
:101CF000090ED926DF503E6E4350D96EDA6A080EBF
:101D0000D926DF503F6E4350D96EDA6A070ED926C6
:101D1000DF50406E4350D96EDA6A060ED926DF5086
:101D2000416E4350D96EDA6A050ED926DF50412440
:101D300040243F243E243D243C243B240001B26F38
:101D4000460EB219D8A412004350D96EDA6ADECF1B
:101D50003BF0DECF3CF0DECF3DF0DECF3EF03F0E7D
:101D60003B143F6E406A416A426A0101501909E121
:101D70005151401806E15251411803E153514218A4
:101D8000D8A41200F29E910E176EFF0E186E3CEC56
:101D900009F0C4EF1DF0F50E176EFF0E186E3CEC47
:101DA00009F00CD0FB0E176EFF0E186E3CEF09F019
:101DB000CE0E176EFF0E186E3CEC09F04350ECEFA0
:101DC0001BF04350D96EDA6AC00EDE143B6EFF0E74
:101DD000DE143C6EFF0EDE143D6EFF0EDE143E6E12
:101DE0003E5033E0080A34E0120A36E0E1D73C50B6
:101DF00005E0010A10E0030A12E0DAD73B5001E1E6
:101E000025D7400A01E143D7C00AD8B41200400ADE
:101E100001E14FD7CDD73B50800ABDE0C9D73B5039
:101E2000400A01E142D7C00A01E121D7C1D73C50A5
:101E30001C0ABEE13B50B6E0BBD73C50010AB8E1FA
:101E40003B50800A01E13CD7B3D73D50D0E0B0D73A
:101E50003D50040AECE0ACD73D50070AEEE0A8D7AD
:101E6000096B0A6B0D6B0E6B086A076A12000E6E27
:101E70000F0120B71ED0210E016E0F0EBBD82FEC24
:101E80001BF00E50D96EFEEC0CF00F01256FD6D86A
:101E9000266FE9D8276FEED8286FC9D8296FC0D828
:101EA0002A6FDAD82B6FB5D82C6FCFD82D6F20873B
:101EB000120010B71ED0110E016E0F0E9BD82FEC22
:101EC0001BF00E50D96EFEEC0CF00F01156FB6D85A
:101ED000166FC9D8176FCED8186FA9D8196FA0D8A8
:101EE0001A6FBAD81B6F95D81C6FAFD81D6F1087AB
:101EF000120000B71ED0010E016E0F0E7BD82FEC22
:101F00001BF00E50D96EFEEC0CF00F01056F96D849
:101F1000066FA9D8076FAED8086F89D8096F80D827
:101F20000A6F9AD80B6F75D80C6F8FD80D6F00871A
:101F300012000E01B0B71ED0B10E016E0E0E5AD8AF
:101F40002FEC1BF00E50D96EFEEC0CF00E01B56FAD
:101F500075D8B66F88D8B76F8DD8B86F68D8B96F95
:101F60005FD8BA6F79D8BB6F54D8BC6F6ED8BD6FCD
:101F7000B0871200C0B71ED0C10E016E0E0E3AD847
:101F80002FEC1BF00E50D96EFEEC0CF00E01C56F5D
:101F900055D8C66F68D8C76F6DD8C86F48D8C96F95
:101FA0003FD8CA6F59D8CB6F34D8CC6F4ED8CD6FCD
:101FB000C0871200D0B71200D10E016E0E0E1AD8D3
:101FC0002FEC1BF00E50D96EFEEC0CF00E01D56F0D
:101FD00035D8D66F48D8D76F4DD8D86F28D8D96F95
:101FE0001FD8DA6F39D8DB6F14D8DC6F2ED8DD6FCD
:101FF000D0871200026E0E50D96EDA6ADECF03F07F
:10200000DECF04F0DECF05F0DECF06F00DC007F026
:1020100012000E50D96EDA6A0B0ED926DF5012006C
:102020000E50D96EDA6A090ED926DF5012000E5012
:10203000D96EDA6A080ED926DF5012000E50D96E1A
:10204000DA6A050ED926DF5012000E50D96EDA6A10
:102050000C0ED926DF5012000E50D96EDA6A0A0E25
:10206000D926DF5012000E50D96EDA6A060ED92634
:10207000DF5012000E50D96EDA6A070ED926DF50F3
:102080001200176E1750D96EDA6AC00EDE14136E86
:10209000FF0EDE14146EFF0EDE14156EFF0EDE143E
:1020A000166E96D0010E016F010C015114E017500D
:1020B0007AEC1DF00F6E040E0019010ED8B4000E5C
:1020C0000F1402E0010E006F016BACEC12F0D8ECC3
:1020D00022F084EC24F01750D96EFEEC0CF00DE1E8
:1020E0001750F3EC0CF0020E0001BA6F09C1BBF0FF
:1020F00001010A510001BC6F54D0175063EC13F07A
:10210000DF64010C040E0101001927E017507AEC7E
:102110001DF0000926E04F51800A750F04E24F2B95
:1021200081EC24F01ED01750D96EDA6A060ED9263B
:10213000DF50106E0F6A1750D96EDA6A050ED92675
:10214000DF500F24096F000E10200A6F010E006F80
:102150006EEC24F0280E4E6F04D0096B0A6B0D6BE9
:102160000E6B01010ABF07D0040E0A5D04E3030EE3
:102170000A6F096912000AAF12000905FC0E0A591C
:10218000D8B01200FC0E0A6F010E096F010C175037
:10219000D96EFEEC0CF00AE11750F3EC0CF068EC91
:1021A00013F0010E0D6EB60E37EF0FF01750D96E0B
:1021B000FEEC0CF0D8B4120017505CEC13F0026A7D
:1021C000050E016E47C103F0D8EC22F084EF24F035
:1021D00013C00FF014C010F015C011F016C012F0AB
:1021E0001250020AD8A412001CD0105006E0010AB6
:1021F00011E0030AD8A4120012D00F5001E155D704
:10220000400A01E14FD7C00A01E14FD7400AD8A4E4
:102210001200BDD70F50400AD8A4120046D70F5065
:10222000FBD71150070AD8A41200DFD7E00ED76EF3
:10223000CF0ED66E5C2A000E5D225E225F22F294E3
:1022400041EC19F0F7EC23F05CB03BD001014C05F8
:1022500007E1E5EC1BF00D6A0C6A030EE1EC1CF0E3
:1022600001014C51D8A44C074C5103E1006B81ECA7
:1022700024F001014D050BE1086A320E076E096A70
:102280000B6A0A6E0D6A0C6A010EE1EC1CF001018A
:102290004D51D8A44D074D5103E1006B81EC24F062
:1022A00001014E51D8A44E074E050BE14F6B096B4F
:1022B0000A6B0D6B0E6B81EC24F0086A076ACCEC9C
:1022C00014F05CC00EF05DC00FF05EC010F05FC097
:1022D00011F0050E126E136A146A156AF2EC20F002
:1022E0000E500F10101011100EE14FEC24F02BC007
:1022F00013F12CC014F128EC1FF029C019F12AC0E9
:102300001AF167EC1FF05CC00EF05DC00FF05EC00C
:1023100010F05FC011F00A0E126E136A146A156A8B
:10232000F2EC20F00E500F1010101110D8B40DEC7C
:102330001EF05CC00EF05DC00FF05EC010F05FC01C
:1023400011F0140E126E136A146A156AF2EC20F082
:102350000E500F101010111011E101014C5106E147
:10236000096B0A6B086A076ACCEC14F0465105E168
:10237000A7EC19F045C146F101D046075CC00EF04C
:102380005DC00FF05EC010F05FC011F0640E126E01
:10239000136A146A156AF2EC20F00E500F10101038
:1023A000111006E153EC21F029C005F12AC006F115
:1023B0005CC00EF05DC00FF05EC010F05FC011F0A9
:1023C000E80E126E030E136E146A156AF2EF20F017
:1023D000176E1750D96EDA6AC00EDE14136EFF0E38
:1023E000DE14146EFF0EDE14156EFF0EDE14166E74
:1023F00083D0080E0119D8B41200040E001902E0AF
:10240000080E016FA9D8D8EC22F084EC24F0030E5A
:1024100001013C6FE80E3B6F3E6B640E3D6F406BFD
:102420003F6F336B346B356B366B1200090E016FE7
:10243000090C1750D96EFEEC0CF006E11750F3ECC6
:102440000CF052EC13F041D0175063EC13F0DF6442
:10245000010C040E001914E01750D96EDA6A060E4A
:10246000D926DF50106E0F6A1750D96EDA6A050E42
:10247000D926DF500F24156F000E1020166F02D0E2
:10248000156B166B16BF0AD0990E155D3A0E1659CC
:1024900005E33A0E166F980E156F980C16AF1200E2
:1024A000680E155DC50E1659D8B01200C50E166F10
:1024B000680E156F680C1750D96EFEEC0CF00AE12F
:1024C0001750F3EC0CF068EC13F0010E0D6EB60E25
:1024D00037EF0FF01750D96EFEEC0CF0D8B41200A5
:1024E00017505CEC13F0026A050E016E47C103F051
:1024F000D8EC22F084EF24F013C00FF014C010F0D9
:1025000015C011F016C012F01250020AD8A4120021
:102510001ED01050080A06E0010A11E0030AD8A4F0
:10252000120012D00F5001E164D7400A01E17ED7BA
:10253000C00A01E17ED7400AD8A41200BCD70F50D0
:10254000800AD8A4120075D70F50400AFAD711504C
:10255000070AD8A41200DDD7026A030E016E0151EA
:10256000FC0B036E1200176E1750D96EDA6AC00E9C
:10257000DE14136EFF0EDE14146EFF0EDE14156EE5
:10258000FF0EDE14166E61D0080E0119D8B41200C9
:10259000040E0019D8B41200080E016F080C090EC1
:1025A000016F090C1750D96EFEEC0CF005E11750C5
:1025B000F3EC0CF077D83CD0175085D8DF64010CD1
:1025C000040E001914E01750D96EDA6A060ED926E7
:1025D000DF50106E0F6A1750D96EDA6A050ED926D1
:1025E000DF500F24156F000E1020166F02D0156BF0
:1025F000166B16BF08D01505040E165904E3030E1A
:10260000166F1569120016AF12001505FC0E16594B
:10261000D8B01200FC0E166F010E156F010C17508A
:10262000D96EFEEC0CF009E11750F3EC0CF050D829
:10263000010E0D6EB60E37EF0FF01750D96EFEEC8F
:102640000CF0D8B41200175037D013C00FF014C0DC
:1026500010F015C011F016C012F01250020AD8A4E2
:1026600012001BD01050080A06E0010A0EE0030A0F
:10267000D8A412000FD00F5087E0400A90E0C00AA3
:1026800091E0400AD8A41200CAD70F50800AD8A4FB
:10269000120088D70F50400AFAD71150070AD8A461
:1026A0001200E0D7020E0001BA6F15C1BBF00101A4
:1026B00016510001BC6F1200D96EDA6A050ED926D8
:1026C000DF50476F1200D96EDA6A040ED926010C6A
:1026D000020E0001BA6F47C1BBF0020C0001736B20
:1026E000020E726FBBEC23F074EC24F088D8BBECC4
:1026F00023F08FD8BBEC23F09AD8BBEC23F090D812
:10270000BBEC23F00101036F500E4C6F096B0A6B99
:102710000D6B0E6B010E456F45C146F1700ED31265
:102720009B8C4E6B8EEC20F00001776B766B1EEC71
:1027300014F001014C6B0001736B640EA7EC23F0E5
:102740002EEC1DF0776B766B1EEC14F0736B020EA3
:10275000726FBBEC23F074EC24F051D8BBEC23F087
:1027600058D8BBEC23F063D8BBEC23F059D8BBECB2
:1027700023F00101036F490E0001886FFF0E896F7E
:1027800055EC06F0ED0E886FFE0E896FAD0E8A6F68
:10279000FF0E8B6F8D6B010E8C6F8F6B070E8E6F24
:1027A000C7EC23F072C090F073C091F0936B926B02
:1027B000030E736FFD0E726FBBEC23F00001946F7C
:1027C000956B030E736FFE0E726FBBEC23F000016E
:1027D000966F976B55EC06F06F0E886FFF0E896F42
:1027E000F0CE8AF08B6BF1CE8CF08D6BF2CE8EF04A
:1027F0008F6BF3CE90F0916B55EC06F0FFD7010193
:10280000506F516B526B536B0001736B030E726F01
:10281000030C0101016F0001736B040E726F040C55
:102820000101476F0001736B060E726F060C010108
:10283000026F0001736B050E726F050CBBAE06D004
:10284000A1D8BBB87981BBBA798309D09BD8BBB872
:102850007981BBBA7983796D7A1FD8B07A2B01015F
:1028600002AD05D00001796D7A1FD8B07A2B000136
:102870007651771146E07651795D726F77517A59CA
:10288000736F50EC23F073BF20D0735103E1790EC6
:10289000725D1BE37951765D7751800A786F7A51CA
:1028A000800A785904E3780E7927000E0CD076510F
:1028B000795D7A51800A786F7751800A785909E3F7
:1028C000880E7927FF0E7A2304D076C079F077C07E
:1028D0007AF07ABF07D07929030E7A5903E3030E01
:1028E0007A6F79697AAF09D0020E795DFC0E7A5958
:1028F00004E2FC0E7A6F010E796F79C076F07AC02F
:1029000077F0010102AD05D00001766D771FD8B0D8
:10291000772B000177AF0AD0766D771FD8B0772B71
:10292000BB9EBB84BB860A0E8A120DD077BF06D031
:10293000775102E1760502E3BB8EF3D7010102ABCA
:1029400002D0BB94BB9676C078F0010E00017817D8
:10295000783BBB507819EF0B7819BB6E773577331E
:10296000763376C078F0010E7817783B7847BB5005
:102970007819DF0B7819BB6E77357733763376C0ED
:10298000BCFF1200BCCF79F07A6BD89079377A37D8
:10299000D89079377A371200BBAE06D09AD8BBB838
:1029A0000A80BBBA0A8209D094D8BBB80A80BBBAE5
:1029B0000A820A6C0B1ED8B00B2A010102AD04D0AA
:1029C0000A6C0B1ED8B00B2A0750081046E00750BF
:1029D0000A5C016E08500B58026E64EC23F002BED4
:1029E00020D0025003E1790E015C1BE30A50075C22
:1029F0000850800A096E0B50800A095804E3780ECB
:102A00000A26000E0CD007500A5C0B50800A096E93
:102A10000850800A095809E3880E0A26FF0E0B2287
:102A200004D007C00AF008C00BF00BBE07D00A287C
:102A3000030E0B5803E3030E0B6E0A680BAE09D0AE
:102A4000020E0A5CFC0E0B5804E2FC0E0B6E010E2B
:102A50000A6E0AC007F00BC008F002AD04D0076C84
:102A6000081ED8B0082A08AE0AD0076C081ED8B0D5
:102A7000082ABB9EBB84BB860A0E8A120CD008BEF5
:102A800006D0085002E1070402E3BB8EF3D702AB85
:102A900002D0BB94BB9607C009F0010E0916093A93
:102AA000BB500918EF0B0918BB6E08340832073207
:102AB00007C009F0010E0916093A0946BB5009186A
:102AC000DF0B0918BB6E08340832073207C0BCFFA1
:102AD0001200BCCF0AF00B6AD8900A360B36D89099
:102AE0000A360B361200176E1750D96EDA6AC00E0E
:102AF000DE14136EFF0EDE14146EFF0EDE14156E60
:102B0000FF0EDE14166E65D0080E0119D8B412003F
:102B1000040E0019D8B41200080E016F080C090E3B
:102B2000016F090C1750D96EFEEC0CF006E117503E
:102B3000F3EC0CF052EC13F03ED0175063EC13F0B2
:102B4000DF64010C040E001914E01750D96EDA6A24
:102B5000060ED926DF50106E0F6A1750D96EDA6A4A
:102B6000050ED926DF500F24156F000E1020166FAA
:102B700002D0156B166B16BF08D01505040E16593A
:102B800004E3030E166F1569120016AF1200150547
:102B9000FC0E1659D8B01200FC0E166F010E156F00
:102BA000010C1750D96EFEEC0CF00AE11750F3EC53
:102BB0000CF068EC13F0010E0D6EB60E37EF0FF04F
:102BC0001750D96EFEEC0CF0D8B4120017505CEF21
:102BD00013F013C00FF014C010F015C011F016C0A0
:102BE00012F01250020AD8A412001BD01050080A8A
:102BF00006E0010A0EE0030AD8A412000FD00F501D
:102C000083E0400A8CE0C00A8DE0400AD8A412009C
:102C1000C8D70F50800AD8A4120084D70F50400A9A
:102C2000FAD71150070AD8A41200E0D7176E175030
:102C3000D96EDA6AC00EDE14136EFF0EDE14146E47
:102C4000FF0EDE14156EFF0EDE14166E65D0080E34
:102C50000119D8B41200040E0019D8B41200080EDD
:102C6000016F080C090E016F090C1750D96EFEECAC
:102C70000CF006E11750F3EC0CF052EC13F03ED0E0
:102C8000175063EC13F0DF64010C040E001914E01C
:102C90001750D96EDA6A060ED926DF50106E0F6A09
:102CA0001750D96EDA6A050ED926DF500F24156F3A
:102CB000000E1020166F02D0156B166B16BF08D0D1
:102CC0001505040E165904E3030E166F156912005C
:102CD00016AF12001505FC0E1659D8B01200FC0EE6
:102CE000166F010E156F010C1750D96EFEEC0CF02B
:102CF0000AE11750F3EC0CF068EC13F0010E0D6EC6
:102D0000B60E37EF0FF01750D96EFEEC0CF0D8B4BA
:102D1000120017505CEF13F013C00FF014C010F046
:102D200015C011F016C012F01250020AD8A41200F9
:102D30001BD01050080A06E0010A0EE0030AD8A4CE
:102D400012000FD00F5083E0400A8CE0C00A8DE0E3
:102D5000400AD8A41200C8D70F50800AD8A4120085
:102D600084D70F50400AFAD71150070AD8A412008E
:102D7000E0D7186E85D80F6E0FC010F0116A126A76
:102D8000136A5051101809E15151111806E15251BE
:102D9000121803E153511318D8A412001850D96E19
:102DA000DA6A0C0ED926DF500F6E1850D96EDA6A27
:102DB0000B0ED926DF50106E1850D96EDA6A0A0E43
:102DC000D926DF50116E1850D96EDA6A090ED9264D
:102DD000DF50126E1850D96EDA6A080ED926DF500D
:102DE000136E1850D96EDA6A070ED926DF50146EAA
:102DF0004ED8156E45D815241424132412241124FA
:102E000010240F24176E460E1718D8A412003FD8AE
:102E1000506F516B526B536B1850D96EDA6AC00EFB
:102E2000DE140F6EFF0EDE14106EFF0EDE14116E38
:102E3000FF0EDE14126E50510F10136E5151101010
:102E4000146E52511110156E53511210166E185007
:102E5000D96EDA6A13C0DEFF14C0DEFF15C0DEFFD4
:102E600016C0DEFF026A020E016E50C103F0D8ECFC
:102E700022F084EC24F0010E0D6E180E37EF0FF0E7
:102E80001850D96EDA6A050ED926DF501200185094
:102E9000D96EDA6A060ED926DF50120000018A6F59
:102EA000800E6F6E6E38E832070B040AF9E1100EDF
:102EB0000E0165D83F0E00017E6F7F6B80691F0E8B
:102EC000816F010E826F000E0FEC23F0000E8A2539
:102ED000866F876B000E8723886B070E8823896BAC
:102EE000020E892386C07EF087C07FF088C080F004
:102EF00089C081F0010E826F000E81EC21F03F0E3F
:102F00007E6F7F6B80698169010E826F000E0FEC0E
:102F100023F07E697F6980698169010E826F0FEC01
:102F200023F0000E8A253BD81A0E8123010E826FF2
:102F3000020E81EC21F0000E8A2531D8020E812389
:102F4000010E826F000E81EC21F07F0E7E6F1C0E51
:102F50007F6F040E806F080E816F010E826F81EC0F
:102F600021F0070E0E01466F476BC40E796F7A6928
:102F70007B696F6A6E38E832070BFBE119D0716F1D
:102F8000320E726F540E736F760E746F980E756FEB
:102F9000BA0E766FDC0E776FFE0E786FFE0C7E6FCA
:102FA0007F6B000E7F23806B070E8023816B1200E6
:102FB000606A0F01306B7882768212000101000591
:102FC0006DE10ABF07D00929030E0A5903E3030E76
:102FD0000A6F09690AAF09D0020E095DFC0E0A5991
:102FE00004E2FC0E0A6F010E096F47512FE00951F0
:102FF0000D5D0E51800A116E0A51800A115805E2CA
:1030000047510D27000E0E230DD00D51095D0A51B9
:10301000800A116E0E51800A115804E247510D5F6B
:10302000000E0E5B4751116E126A09510D5D016E63
:103030000A510E59026E64EC23F01150015C0250EB
:10304000800A136E1250800A135804E209C10DF170
:103050000AC10EF10EBF07D00D29030E0E5903E36E
:10306000030E0E6F0D690EAF09D0020E0D5DFC0E42
:103070000E5904E2FC0E0E6F010E0D6F0DEC1EF0EA
:1030800001C007F002C008F0CCEC14F00DEC1EF00B
:1030900001C00FF002C010F090EF1BF0086A076A41
:1030A000CCEC14F0106A0F6A90EF1BF0645121E130
:1030B00060C0D9FF61C0DAFFDF50656FD890653717
:1030C000D8906537D8906535686F56D8D8906533F5
:1030D000662FFCD76551696F47D8656F050E666F1F
:1030E000D8906533662FFCD7655168136A6B6B6B9C
:1030F0002ED060C0D9FF61C0DAFFDF5046D86B6FB9
:103100003BD8D8906537662FFCD765516A6F676BDF
:103110002BD802E0010E676F6739E8461F0B6A1370
:1031200020EE02F06051D9266151DA22DF50696F3A
:103130001BD82BD81C0B6A1317D8030B6A1320EE6D
:1031400003F06051D9266151DA22DF50686F62C006
:10315000D9FF63C0DAFF68C0DEFF69C0DEFF6AC066
:10316000DEFF6BC0DEFF120020EE01F06051D926B9
:103170006151DA22DF50120060C0D9FF61C0DAFF6E
:10318000DF50656F050E666F050C656FD89065336F
:10319000D8906533D89065311200016E5B500D0DEB
:1031A000000EF324D96E020EF420DA6E0150E16EA7
:1031B000E26ADECFE6FFDECFE6FFDECFE6FFDECF60
:1031C000E6FF5B50B3EC0BF00150E16EE26A040ED7
:1031D000E126DFCFE7FF5B50BBEC0BF00150E16E67
:1031E000E26A050EE126DFCFE7FF5B50ABEC0BF0A8
:1031F0000150E16EE26A060EE126DFCFE7FF5B5089
:10320000A3EC0BF00150E16EE26A070EE126DFCF7E
:10321000E7FF5B50CBEC0BF00150E16EE26A080E69
:10322000E126DFCFE7FF5B50C3EC0BF00150E16E0E
:10323000E26A090EE126DFCFE7FF5B50DBEC0BF023
:103240000150E16EE26A0A0EE126DFCFE7FF5B5034
:10325000D3EC0BF00150E16EE26A0B0EE126DFCFFA
:10326000E7FF5B50E3EC0BF00150E16EE26A0C0EFD
:10327000E126DFCFE7FF5B2A0F0E5B16B007B01722
:103280000F0C0001A651A71114E0A607D8A0A707AC
:10329000A651A7110EE1030E086E840E076E096A8F
:1032A000030E0B6E840E0A6E000E0D6A0C6AE1ECC2
:1032B0001CF0B45105E1B35103E18B9A8B981200D5
:1032C000AE51AF110DE1AC07D8A0AD07AC51AD11B7
:1032D00034E1AAC0AEF0ABC0AFF0B4C0B5F02DD0B1
:1032E000AC51AD110DE1AE07D8A0AF07AE51AF1193
:1032F00024E1A8C0ACF0A9C0ADF0B3C0B5F01DD0BA
:10330000A8C0ACF0A9C0ADF0AE6BAF6B16D08B9A75
:103310008B9812008B8A8B9812008B9A8B881200E4
:10332000010E8BA8000E0F6E010E8BAA000E0F1A55
:10333000D8B48B7A8B7A8B781200B551E8E0010A09
:10334000ECE0030AE7E0010AD8A41200E9D723D889
:1033500048EC21F027D80D6EB60E37EC0FF021EEB9
:1033600050F0000EDE100001B66F280E48EC21F080
:1033700030D80D6EB60E37EC0FF021EE50F0000E87
:10338000DE100001B66F2C0E48EC21F033D80D6E24
:10339000B60E37EF0FF021EE50F0000EDE100001F8
:1033A000B66F240C00C1BBF005C1BCF00101065191
:1033B0000001BD6F02C1BEF00DC1BFF001010E5191
:1033C0000001C06F19C1C1F001011A510001C26FA3
:1033D000010C48C1BBF0010149510001BC6F4AC159
:1033E000BDF001014B510001BE6FBF6BC06BC16BE3
:1033F000C26B010C23C1BBF024C1BCF025C1BDF0E0
:1034000026C1BEF01FC1BFF020C1C0F021C1C1F074
:1034100022C1C2F0010C12341334186E185005E1A9
:10342000106A116A126A136A1200163417341E6E7B
:103430001E5005E1106A116A126A136A12001E50CA
:103440007B0F182613C01EF017501E1A800E1E1672
:10345000128E168E000E1716196A1A6A1B6A1C6ADB
:10346000070E1D6E10B029D831D814361536163611
:1034700017361D2EF7D7110E1D6E10B01ED826D888
:103480001C321B321A3219321D2EF7D719C001F027
:103490001AC002F01BC003F01CC004F018C005F0F5
:1034A0001EC006F0CEEC1AF001C010F002C011F000
:1034B00003C012F004C013F0120014501926155066
:1034C0001A2216501B2217501C221200D8901332B9
:1034D000123211321032D8901200785113E174C0B8
:1034E00079F075C07AF076C07BF077C07CF0040E7E
:1034F00001D04ED8E82EFDD73ED87439E846E00B0F
:10350000DF6E120074C079F075C07AF076C07BF07F
:1035100077C07CF0160E01D03BD8E82EFDD72BD813
:1035200076C079F0030E791774C07AF075C07BF01D
:1035300076C07CF077C07DF00E0E05D0D8907D333C
:103540007C337B337A33E82EF9D77A51E00B79114B
:103550000809DF6E20EE02F07251D9267351DA228B
:1035600075C0DFFF20EE03F07251D9267351DA22C5
:1035700074C0DFFF1200795172C0D9FF73C0DAFF47
:10358000DF6E20EE01F07251D9267351DA2212005B
:10359000D8907C337B337A3379331200055005E0C1
:1035A000015002100310041007E1016A026A036A65
:1035B000046A1200052A4DD8076A086A096AFE0ED5
:1035C00004140A6E0750081009100A1008E0F2D718
:1035D000052A012A000E0222032204223AD8076A91
:1035E000086A096A04500A6E0750081009100A1088
:1035F00007E0EED70506D8900136023603360436CA
:1036000003BE03D0020E0560F5D705B002D07F0ED1
:103610000316D890053205C007F0086A096A0A6ADD
:1036200007C00AF0096A086A076A075001120850C1
:103630000212095003120A5004120650D8A4048E34
:1036400001C001F002C002F003C003F004C004F0A6
:103650001200D890043203320232013212000750B5
:1036600013E103C008F004C009F005C00AF006C069
:103670000BF0040E01D04ED8E82EFDD73ED803380B
:10368000E846E00BDF6E120003C008F004C009F04A
:1036900005C00AF006C00BF0160E01D03BD8E82E8C
:1036A000FDD72BD805C008F0030E081603C009F09B
:1036B00004C00AF005C00BF006C00CF00E0E05D0D9
:1036C000D8900C320B320A320932E82EF9D7095061
:1036D000E00B08100809DF6E20EE02F00150D92639
:1036E0000250DA2204C0DFFF20EE03F00150D92699
:1036F0000250DA2203C0DFFF1200085001C0D9FFD8
:1037000002C0DAFFDF6E20EE01F00150D926025030
:10371000DA221200D8900B320A3209320832120033
:103720000F5010100EE10B510C1106E04ED8000E98
:103730000D6A0C6AE1EC1CF00FC00BF110C00CF12B
:1037400012000FC00BF110C00CF10FC001F010C03F
:1037500002F0046A020E036EA5EC1FF001C00FF028
:1037600002C010F0040E0019D8B4120010BE17D019
:10377000105002E10F0413E30F28076E000E102013
:10378000086E096A0F5000080A6E1050D8A0E82A87
:1037900002080B6E0D6A0C6A010EE1EF1CF010AE10
:1037A00012000F500108076E1050D8A0E82A000838
:1037B000086E000E096A0F240A6E020E10200B6EAE
:1037C0000D6A0C6A020EE1EF1CF0086A640E076EC7
:1037D000096A0B6A0A6E640C3A6E800E176EFF0E51
:1037E000186E5CC019F05DC01AF05EC01BF05FC0BF
:1037F0001CF03A50D96EDA6AC00EDE141D6EFF0E50
:10380000DE141E6EFF0EDE141F6E1F0EDE14206E01
:103810003A50D96EDA6ADECF21F0DECF22F0DECF69
:1038200023F0DECF24F03A50D96EFEEC0CF0256E7A
:10383000266A3CEC09F0386A396A11D08D0E176E91
:10384000FF0E186E3A503824D96EDA6A050ED92662
:10385000DF50196E1A6A3CEC09F0384A392A3A509E
:10386000D96EFEEC0CF0356E366A3550385C395046
:10387000800A376E3650800A3758E0E37D0E176EA7
:10388000FF0E186E3CEF09F00001866F800E6F6E20
:10389000948C948E02D0800E6F6E6E38E832070BD7
:1038A000040AF9E1800E726EE00E0E017D6F0AD0FF
:1038B000930E05D08F0E03D0830E01D0810E06EC3F
:1038C0001EF00AD000018651F3E0010AF3E0030A7A
:1038D000F3E0010AF3E0F0D7100EBFEC17F0000E92
:1038E00000011AD8000E0FEC23F0000E15D80FECD3
:1038F00023F07E6B7F6B806B816B010E826F000EFD
:1039000081EC21F0010E0E01466F6F6A6E38E832CD
:10391000070BFBE1D8EF17F07E6F7F6F806F816F31
:10392000010E826F010C21342234286E285005E1EB
:103930001F6A206A216A226A12001FC023F020C079
:1039400024F021C025F022C026F0200E05D0D8900A
:103950002632253224322332E82EF9D72350276E1F
:10396000218E226A960E285E28AE0CD02850800A3E
:10397000970FDEE3D8902232213220321F32283EC8
:10398000F9D70CD01F0E286407D0D2D7D8901F3695
:1039900020362136223628062850F8E1275008E044
:1039A000221E211E201E1F6C000E202221222222F8
:1039B0001FC01FF020C020F021C021F022C022F043
:1039C00012000E6E0C500001A61916E10D50A71939
:1039D00013E10E50B31910E10950B4190DE107506D
:1039E000A8190AE10850A91907E10A50AA1904E127
:1039F0000B50AB19D8B41200310E0C5C750E0D587B
:103A000004E3750E0D6E300E0C6E0CC0A6F00DC0EA
:103A1000A7F0E30E075C040E085804E3040E086EDA
:103A2000E20E076EE30E0A5C040E0B5804E3040E6C
:103A30000B6EE20E0A6E0EC0B3F009C0B4F007C000
:103A4000A8F008C0A9F00AC0AAF00BC0ABF0A8C04B
:103A5000ACF0A9C0ADF0AE6BAF6B1200796F7751CF
:103A6000A61916E17851A71913E17951B31910E19C
:103A70007451B4190DE17251A8190AE17351A919D1
:103A800007E17551AA1904E17651AB19D8B41200B7
:103A9000310E775D750E785904E3750E786F300E30
:103AA000776F77C0A6F078C0A7F0E30E725D040EC2
:103AB000735904E3040E736FE20E726FE30E755DCB
:103AC000040E765904E3040E766FE20E756F79C02A
:103AD000B3F074C0B4F072C0A8F073C0A9F075C0A0
:103AE000AAF076C0ABF0A8C0ACF0A9C0ADF0AE6B48
:103AF000AF6B1200096E3ED00950D96EDA6A0C0E17
:103B0000D926DF50016E0950D96EDA6A0B0ED9261C
:103B1000DF50026E0950D96EDA6A0A0ED926DF50DC
:103B2000036E0950D96EDA6A090ED926DF50046E89
:103B30000950D96EDA6A080ED926DF50056E1DD8F5
:103B4000066E0950D96EDA6A060ED926DF50076E66
:103B50000950D96EDA6A050ED926DF5007240624EB
:103B600005240424032402240124086E085001E1E2
:103B7000010C000C02D8C0E0000C0950D96EDA6AC2
:103B8000070ED926DF5012009F0E176EFF0E186E1B
:103B90003CEC09F0700ED3129B8C800E6F6EC00E41
:103BA000946E550E8B6E81EC24F002D0800E6F6EF9
:103BB0006E38E832070B040AF9E1810E27D8726AE1
:103BC0007D6B716B726B736B746B756B766B776BF4
:103BD000786BE069E169E269E369F86BF96BFA6BAC
:103BE000FB6B01D06F6A6E38E832070BFBE1400EC9
:103BF000606E0F01306FAA0E8B6E320E176EFF0EC5
:103C0000186E3CEC09F001EF00F012000E01436F5A
:103C1000B80E446F050E456F050C80AE03D0010150
:103C2000028102D00101029180AC02D0028301D056
:103C3000029302AD0FD021EE0DF0DECF03F0DDCF09
:103C400004F0031E041E034A042A03C005F004C046
:103C500006F004D00DC105F00EC106F002A520D07B
:103C600002A70BD006BE11D0065002E105040DE3F9
:103C700080AE0BD0016A026A120006BE06D0065062
:103C800002E1050402E380AEF5D702A905D006AE35
:103C900007D080BCEFD704D006AE02D080ACEAD704
:103CA0000DC101F00EC102F012000F6E0F50F3ECC7
:103CB0000CF00F50D96EFEEC0CF00001BA6F0F50F3
:103CC000D96EDA6A050ED926DF50BB6F0F50D96E58
:103CD000DA6A060ED926DF50BC6F0F50D96EDA6A49
:103CE000070ED926DF50BD6F0F50D96EDA6A080E65
:103CF000D926DF50BE6F0F50D96EDA6A090ED92669
:103D0000DF50BF6F0F50D96EDA6A0A0ED926DF5026
:103D1000C06F0F50D96EDA6A0B0ED926DF50C16F13
:103D20000F50D96EDA6A0C0ED926DF50C26F010E21
:103D30000D6EB60E37EF0FF021EE50F0000EDE10D4
:103D40000001B66F380E48EC21F0026A400E016E99
:103D500003EC24F00001BB6F026A410E016E03EC1C
:103D600024F00001BC6F026A420E016E03EC24F0E5
:103D70000001BD6F026A430E016E03EC24F00001E6
:103D8000BE6F026A440E016E03EC24F00001BF6FA7
:103D9000026A450E016E03EC24F00001C06F026A56
:103DA000460E016E03EC24F00001C16F026A470E5B
:103DB000016E03EC24F00001C26F010E0D6EB60E11
:103DC00037EF0FF021EE50F0000EDE100001B66F5D
:103DD000440E48EC21F0026A380E016E03EC24F028
:103DE0000001BB6F026A390E016E03EC24F0000182
:103DF000BC6F026A3A0E016E03EC24F00001BD6F45
:103E0000026A3B0E016E03EC24F00001BE6F026AF1
:103E10003C0E016E03EC24F00001BF6F026A3D0E00
:103E2000016E03EC24F00001C06F026A3E0E016EC9
:103E300003EC24F00001C16F026A3F0E016E03EC37
:103E400024F00001C26F010E0D6EB60E37EF0FF0B9
:103E500025EC24F001C02FF002C030F030AE02D0CB
:103E60002F6A306A2FEC24F001C02DF002C02EF032
:103E70002EAE02D02F6A306A146A156A880E166E4A
:103E8000400E176E2D502F5C0B6E2E5030580C6E5E
:103E9000BBEC22F00BC010F00CC011F00DC012F002
:103EA0000EC013F00BEC1AF010C01FF011C020F080
:103EB00012C021F013C022F093EC1CF01FC02BF0B5
:103EC00020C02CF02BC029F02CC02AF012000101D8
:103ED0004D510BE1086A076ACCEC14F0086A320E07
:103EE000076E096A0B6A640E0BD04C5112E1086A26
:103EF000076ACCEC14F0086A640E076E096A0B6A54
:103F00000A6E0D6A0C6A030EE1EF1CF0120012003B
:103F10001200015102E1DEEF17F0010AD8B41200DD
:103F2000030AF4E0010AD8B41200070AF0E0010A1B
:103F3000D8B41200030AECE0010AD8B412000F0A48
:103F400002E111EF0DF0010A1200066A04AE06D07C
:103F5000036C041ED8B0042A010E066E02AE06D011
:103F6000016C021ED8B0022A010E061A076A086AFE
:103F7000035004101BE0010E056E04D0D8900336E8
:103F80000436052A04AEFAD7D8900736083603500F
:103F9000015C0450025805E30350015E0450025ACC
:103FA0000780D89004320332052EEED7065004E085
:103FB000076C081ED8B0082A07C001F008C002F03C
:103FC00012007A6B7B6B7C6B7D6B7651771178116D
:103FD000791129E0010E7E6F06D0D89076377737B9
:103FE000783779377E2B79AFF8D7D8907A377B3707
:103FF0007C377D377651725D77517359785174599A
:104000007951755909E37651725F7751735B785135
:10401000745B7951755B7A81D890793378337733D3
:1040200076337E2FE2D77AC072F07BC073F07CC00B
:1040300074F07DC075F01200096A0A6A0B6A0C6A96
:10404000055006100710081029E0010E0D6E06D06D
:10405000D89005360636073608360D2A08AEF8D74A
:10406000D89009360A360B360C360550015C0650DE
:104070000258075003580850045809E30550015EE0
:104080000650025A0750035A0850045A0980D89023
:1040900008320732063205320D2EE2D709C001F090
:1040A0000AC002F00BC003F00CC004F01200176E3F
:1040B0001750D96EDA6AC00EDE14136EFF0EDE14CE
:1040C000146EFF0EDE14156EFF0EDE14166E0CD08D
:1040D0001750F3EC0CF0010E0001BA6F00C1BBF0F9
:1040E0000D6EB60E37EF0FF013C00FF014C010F0C6
:1040F00015C011F016C012F01250020AD8A4120016
:1041000008D01050140AD8A412000F50D8A41200DE
:10411000DFD71150070AD8A41200F3D7700ED312BC
:104120009B8C9496829623EC21F0030E44EC1CF0B9
:10413000010150514EEC17F05C6B5D6BF00E5B6F44
:10414000F19E5C6B5D6B94969484928E928C1BECCA
:1041500024F0D3EC23F09DEC23F048EC24F0EBECBE
:1041600023F05CEC24F07DEC24F0DFEC23F0000184
:10417000776B766B1EEC14F0D08EF28CF28EAEEF75
:1041800023F0835184118511861123E0010E876F7E
:1041900006D0D8908337843785378637872B86AF0C
:1041A000F8D783517F5D845180598551815986515B
:1041B000825908E383517F5F8451805B8551815B25
:1041C0008651825BD8908633853384338333872F3F
:1041D000E8D77FC07FF080C080F081C081F082C0CE
:1041E00082F01200125013101410151023E0010E6B
:1041F000166E06D0D8901236133614361536162A97
:1042000015AEF8D712500E5C13500F5814501058BA
:104210001550115808E312500E5E13500F5A1450E7
:10422000105A1550115AD8901532143213321232D6
:10423000162EE8D70EC00EF00FC00FF010C010F011
:1042400011C011F01200CBEC19F022D8D2EC19F009
:104250007E6FB60ED1EC07F021EE50F0000EDE10AE
:104260000001B66F280E14D8E9EC19F07E6FB60E77
:10427000D1EC07F021EE50F0000EDE100001B66F19
:104280002C0E06D8FAEC19F07E6FB60ED1EF07F0BF
:10429000DE10B76F070EDE10B86F020EDE10B96FBA
:1042A000080EBA6F080C010EC26EC282C2B2FED7EF
:1042B0001BD827EC23F00BC010F00CC011F00DC080
:1042C00012F00EC013F00BEC1AF010C01FF011C06A
:1042D00020F012C021F013C022F093EC1CF01FC09C
:1042E00029F020C02AF01200770E146EBE0E156E53
:1042F000BF0E166E3F0E176EC3CF0BF0C4CF0CF07F
:104300003F0C836F0FD0E00E09D0E40E07D0E80E0B
:1043100005D0EC0E03D0F00E01D0F40E846F0E0E1B
:10432000856F0BD08351EFE0010AEFE0030AEFE065
:10433000010AEFE0070AEFE0F0D784C072F085C011
:1043400073F07EC074F07FC075F080C076F081C0DD
:1043500077F082C078F06DEF1AF0106E116A1AD8FB
:104360001F0EDF640BD016D87F0EDF6007D019D880
:1043700011D8DF50036ED8EC22F004D012D8036AB3
:10438000D8EC22F084EC24F0112A070E1164E7D750
:104390009CEF1EF010501124D96EDA6A050ED92652
:1043A000050C400E1124016E026A000E0222000C60
:1043B00021EE50F0000EDE100001B66F300E48EC1A
:1043C00021F0010EBB6F070EBC6F0FEC24F0015003
:1043D000BD6FBE6B030E026EFD0E016E03EC24F08A
:1043E0000001BF6F030E026EFE0E016E03EC24F09F
:1043F0000001C06FC16BC26B010E0D6EB60E37EFC0
:104400000FF0D0C001F0D1C002F0D2C003F0D3C091
:1044100004F06D0E056E4E0E066EC60E076E410E52
:10442000086E4FEC22F001C0D0F002C0D1F003C002
:10443000D2F004C0D3F0390E0001D027300ED123C2
:10444000000ED223D323D2510D6E7F0ED3150E6EE4
:10445000120004AE09D0016C021ED8B0022A031E5D
:10446000D8B0032A800E045608AE09D0056C061E8B
:10447000D8B0062A071ED8B0072A800E0856800E2C
:10448000041A081A0550015C0650025807500358D8
:104490000850045802E2D8901200D8801200096A2D
:1044A0000A6A0B6A0C6A01A008D00550092606505A
:1044B0000A2207500B2208500C22D89005360636E7
:1044C00007360836D89004320332023201320150E6
:1044D000021003100410E7E109C001F00AC002F065
:1044E0000BC003F00CC004F012000F6A0EAE0AD02D
:1044F0000E1E0D1E0C1E0B6C000E0C220D220E2229
:10450000010E0F6E0BC001F00CC002F00DC003F0E5
:104510000EC004F0960E056E0FC006F0CEEC1AF039
:1045200001C00BF002C00CF003C00DF004C00EF08F
:104530001200050EC26EC282C2B2FED774EC21F028
:1045400027EC23F00BC010F00CC011F00DC012F0DE
:104550000EC013F00BEC1AF010C01FF011C020F0C9
:1045600012C021F013C022F093EC1CF01FC029F000
:1045700020C02AF012000F6A0CAE05D00B6C0C1E86
:10458000D8B00C2A0F2A0BC001F00CC002F0036A4D
:10459000046A960E056E0FC006F0CEEC1AF001C04C
:1045A0000BF002C00CF003C00DF004C00EF01200BE
:1045B0000250030B756E01C074FF03C073FF7F9E32
:1045C0007F9C7F84000EF2BE010E046EF29E550E9B
:1045D0007E6EAA0E7E6E7F827FB2FED704B002D0BE
:1045E000F29E01D0F28E7F94120002EE00F0D00E07
:1045F000EE6AE806FDE101EE00F0540EEE6AE80610
:10460000FDE100EEA6F02A0EEE6AE806FDE15F6A23
:104610005E6A5D6A5C6A5B6A00016EEF13F0836F2D
:104620008351F80ED8A4FC0E846F0E0E856F84C0E3
:1046300072F085C073F07EC074F07FC075F080C0EA
:1046400076F081C077F082C078F06DEF1AF00BC081
:1046500001F00CC002F0036A046A960E056E000EAB
:10466000066ECEEC1AF001C00BF002C00CF003C0D5
:104670000DF004C00EF012000001736F0CD0170E85
:1046800056EC24F0170E56EC24F0170E56EC24F0DE
:10469000170E56EC24F073077329D8B41200EFD725
:1046A00073AF0DD072C074F073C075F0741F751FB6
:1046B000744B752B74C072F075C073F0120072C029
:1046C00072F073C073F0120002AE0DD001C003F09F
:1046D00002C004F0031E041E034A042A03C001F0B2
:1046E00004C002F0120001C001F002C002F012008A
:1046F00001500302F3CF05F0F4CF06F0015004029D
:10470000F350062602500302F350062605C001F0BE
:1047100006C002F01200F4CF71F077A205D0500E5F
:1047200001014D6F9AEC0AF071C0F4FF70C0F3FF05
:104730006FC0DAFF6EC0D9FF1100949A94988B8AEB
:104740008B980001736BC80E02D82EEF1DF0726FAC
:10475000746B766B756F786B776B000C01010005DD
:10476000D8A41200949682960A0E3CEC23F082861E
:10477000010E3CEF23F07351030B756E72C074FF92
:104780007F9C7F9E7F8000F000F073501200746B5E
:1047900080BA748182B0748382B27485742B74C0C1
:1047A00072F0736B1200900EA66E240EBA6E938C8C
:1047B000939E080EB96E8A0E7B6E7C6A120079ECAD
:1047C00024F093929394939693984C0EBB6E996AAF
:1047D000800EBC6E800C928403D85D87C28212006A
:1047E000010EC26E300EC16EA50EC06EA50C06D0B5
:1047F000C30ECDEC18F0C30E52EC04F00001B05122
:10480000D8B41200F5D70250030B756E01C074FFC7
:104810007F9C7F9E7F8000F000F073501200036A3F
:1048200080BA038082B0038282B20384032A03C069
:1048300001F0026A1200800ED56EE00ED76ECF0E28
:10484000D66EF294F28AF194CF0C0D0EC26EC28233
:10485000C2B2FED7C3CF01F0C4CF02F01200090EDE
:10486000C26EC282C2B2FED7C3CF01F0C4CF02F083
:10487000120001C0D0F002C0D1F00001D26BD36BA6
:1048800012000001726FA4A8FED772C079FF120057
:104890009280F0EC23F00F015D81C282120099EC4E
:1048A00022F029C02BF02AC02CF01200726F720780
:1048B0007229D8B41200FBD79284F0EC23F05D8506
:1048C000C2821200016E01060128D8B41200FBD783
:1048D000016EA4A8FED701C079FF12000005D8A47C
:1048E00012009496828612000001726F72513F0B83
:1048F0001200070ECA6ECB681200928A94809482CE
:1049000012009496829612007FA21200FDD7010039
:104910000000120012001200FF00FF00FF00FF0065
:10FEA000FF00FF0000010000000A000000640000E5
:10FEB00000E803000010270000A086010040420F68
:10FEC000008096980000E1F50500CA9A3B01000009
:10FED0000010000000000100000010000000000100
:10FEE0000000001000000000010000001053443525
:10FEF000343043202D2025732046572D25642E2590
:10FF0000642048572D25642E256420424C2D2564FD
:10FF10002E25640D0A00756D7077723D20256420D2
:10FF200063706F7765723D25642073703D25640DA5
:10FF30000A000D0A5F5F5F6D6B7374722820424F79
:10FF40004F544C4F41442920000D0A53443534305E
:10FF500043205265626F6F74696E670D0A0030311D
:10FF6000323334353637383961626364656600256B
:10FF7000782025782020257820202578200D0A005B
:10FF8000256C7520256C7820256C7820202578201C
:10FF9000000D0A676F746F426F6F74282920000D7F
:10FFA0000A696E20676F746F426F6F7400466562F6
:10FFB0002031362032303137005359535245535592
:10FFC0004D452000444556515545525920004E4F4D
:10FFD0004E20535953200053595348414C5420004C
:10FFE0005359535253542000286E756C6C290025C8
:10FFF0006C780D0A0053594E4320002E210000005A
:00000001FF
